:0A0DF00000010202030304040505DC
:10080700E4F513F512F511F510C203C200C202C2D6
:10081700011209DF7E007F908E458F46754D00756A
:100827004EA27543007544AC754B00754CDA754F95
:100837000175500890E680E030E70E854347854410
:1008470048854B49854C4A800C854B47854C4885E4
:10085700434985444AEE54E0700302097875140051
:100867007515807E007F908E168F17C3742E9FFF9D
:1008770074019ECF2402CF3400FEE48F0F8E0EF555
:100887000DF50CF50BF50AF509F508AF0FAE0EAD32
:100897000DAC0CAB0BAA0AA909A808C3120F2F505D
:1008A7002AE515250BF582E514350AF58374CDF095
:1008B700E4FAF9F8E50B2401F50BEA350AF50AE93C
:1008C7003509F509E83508F50880C0E4F50BF50AA0
:1008D700F509F508AF0FAE0EAD0DAC0CAB0BAA0AC0
:1008E700A909A808C3120F2F5035AE0AAF0BE51799
:1008F7002FF582E5163EF583E0FDE5152FF582E538
:10090700143EF583EDF0E4FAF9F8EF2401F50BEA6C
:100917003EF50AE93509F509E83508F50880B58592
:10092700144585154674902480FF740034FFFEC378
:10093700E54E9FF54EE54D9EF54DC3E5489FF548BD
:10094700E5479EF547C3E54A9FF54AE5499EF549C0
:10095700C3E5449FF544E5439EF543C3E54C9FF546
:100967004CE54B9EF54BC3E5509FF550E54F9EF583
:100977004FD2E843D82090E668E04409F090E65C5F
:10098700E0443DF0D2AF90E680E020E105D20812C6
:10099700148C90E680E054F7F0538EF8C2033001D0
:1009A7000512056DC20130032912008D5024C203C0
:1009B7001215BC20001690E682E030E704E020E143
:1009C700EF90E682E030E604E020E0E41214EA1259
:0709D7000DFE12145C80C745
:0109DE0022F6
:10056D0090E6B9E070030206491470030206F22406
:10057D00FE700302078724FB700302064314700309
:10058D0002063D147003020631147003020637246F
:10059D000560030207F312173740030207FF90E6C9
:1005AD00BBE024FE602C14604724FD6016146031FE
:1005BD0024067066E54590E6B3F0E54690E6B4F0A6
:1005CD000207FFE54D90E6B3F0E54E90E6B4F0027C
:1005DD0007FFE54790E6B3F0E54890E6B4F0020773
:1005ED00FFE54990E6B3F0E54A90E6B4F00207FF67
:1005FD0090E6BAE0FF121516AA06A9077B01EA4993
:10060D004B600DEE90E6B3F0EF90E6B4F00207FF0D
:10061D0090E6A0E04401F00207FF90E6A0E044015F
:10062D00F00207FF1216B00207FF1217080207FFAC
:10063D0012131B0207FF12169E0207FF12173940F5
:10064D00030207FF90E6B8E0247F602B14603C2482
:10065D000260030206E8A200E433FF25E0FFA202D8
:10066D00E4334F90E740F0E4A3F090E68AF090E693
:10067D008B7402F00207FFE490E740F0A3F090E6E0
:10068D008AF090E68B7402F00207FF90E6BCE0540E
:10069D007EFF7E00E0D3948040067C007D018004C7
:1006AD007C007D00EC4EFEED4F24F0F582740D3E86
:1006BD00F583E493FF3395E0FEEF24A1FFEE34E6DE
:1006CD008F82F583E0540190E740F0E4A3F090E6CB
:1006DD008AF090E68B7402F00207FF90E6A0E044EA
:1006ED0001F00207FF12173B40030207FF90E6B827
:1006FD00E024FE601D240260030207FF90E6BAE0CD
:10070D00B40105C2000207FF90E6A0E04401F0022B
:10071D0007FF90E6BAE0705990E6BCE0547EFF7E8C
:10072D0000E0D3948040067C007D0180047C007D38
:10073D0000EC4EFEED4F24F0F582740D3EF583E492
:10074D0093FF3395E0FEEF24A1FFEE34E68F82F5A3
:10075D0083E054FEF090E6BCE05480FF1313135475
:10076D001FFFE0540F2F90E683F0E04420F00207C6
:10077D00FF90E6A0E04401F0807812173D50739091
:10078D00E6B8E024FE60202402706790E6BAE0B47B
:10079D000104D200805C90E6BAE06402605490E6F9
:1007AD00A0E04401F0804B90E6BCE0547EFF7E005B
:1007BD00E0D3948040067C007D0180047C007D00A8
:1007CD00EC4EFEED4F24F0F582740D3EF583E4936F
:1007DD00FF3395E0FEEF24A1FFEE34E68F82F58323
:1007ED00E04401F0800C120130500790E6A0E04487
:0907FD0001F090E6A0E04480F058
:0108060022CF
:03003300020DFAC1
:040DFA0053D8EF32A9
:1000900012010002000000401816011500000102C4
:1000A00000010A06000200000040010009022E00C3
:1000B000010100A0FA0904000004FF000000070588
:1000C0000102400000070586020002000705020247
:1000D0000002000705810240000009022E00010114
:1000E00000A0FA0904000004FF0000000705010257
:1000F000400000070586024000000705020240009C
:100100000007058102400000040309040E035100AA
:1001100048005900430043004400140351004800C4
:1001200059002D0031003500200020002000000083
:03004300020E00AA
:03005300020E009A
:100E000002161400021688000216720002162C0048
:100E1000021352000213890002008F0002173F00E4
:100E20000217400002174100020F66000210A500E1
:100E30000217420002174300021744000217450040
:100E40000217460002173F0002174700021748002A
:100E50000217490002174A0002174B0002174C0004
:100E600002174D0002173F0002173F0002173F0014
:100E700002174E0002174F000217500002175100D0
:100E800002175200021753000217540002175500B0
:100E90000217560002175700021758000217590090
:100EA00002175A0002175B0002175C0002175D0070
:080EB00002175E0002175F004B
:1014EA0090E682E030E004E020E60B90E682E0300D
:1014FA00E119E030E71590E680E04401F07F147EC0
:0C150A000012129790E680E054FEF022E0
:1015BC0090E682E044C0F090E681F04387010000A1
:0415CC0000000022F9
:10148C0030080990E680E0440AF0800790E680E09E
:10149C004408F07FDC7E0512129790E65D74FFF035
:0F14AC0090E65FF05391EF90E680E054F7F02266
:02151600A90723
:10151800AE4FAF508F828E83A3E064037017AD0186
:1015280019ED7001228F828E83E07C002FFDEC3E46
:09153800FEAF0580DF7E007F009C
:011541002287
:101297008E1E8F1F90E600E054187012E51F240180
:1012A700FFE4351EC313F51EEF13F51F801590E6F7
:1012B70000E05418FFBF100BE51F25E0F51FE51EE2
:1012C70033F51EE51F151FAE1E7002151E4E600575
:0612D7001215D080EE228A
:1015D0007400F58690FDA57C05A3E582458370F92E
:0115E00022E8
:10124800022C1A0002270000023C0000023F03F7AC
:101258000236000002240000022A000001300101C9
:101268003400013300013B00013E00013200022E30
:1012780000000142A0013100013A000129000135B6
:0E12880000C107014100012200013800C1042D
:1009DF0090E6007412F090E6017443F0000000906E
:1009EF00E61074A0F000000000000090E611F00087
:1009FF00000000000090E612F0000000E490E61303
:100A0F00F000000090E61474E0F0000000E490E6BF
:100A1F0015F000000090E6047480F00000007402EE
:100A2F00F00000007406F0000000E4F000000090F9
:100A3F00E60274E6F000000090E60374F8F00000A0
:100A4F000090E670E04440F0000000E490E609F00A
:100A5F0000000053B2FE43B20243B20890E61804FE
:100A6F00F00000007411F000000090E61A7409F015
:100A7F00000000E490E671F090E672F075B4FF7537
:100A8F00B6BF90E65EE04408F0000000E490E68D0B
:100A9F00F090E65EE04404F0000000E490E68FF092
:100AAF00D28112171843B110E4FD7F801211C17F5C
:100ABF00647E001212977D807F801211C1C2057D66
:100ACF000D7F401211C17D787F201211C1E4FD7F8F
:100ADF00101211C1E4FD7F081211C1E4FD7F021253
:100AEF0011C1E4FD7F041211C112171090E67AE0D4
:100AFF0054FEF0E4FD7F9012156D1217601215422F
:100B0F00D2A043B180E4F53A12165B7FC81212DD12
:0F0B1F007DFF7F4212156DE4FD7F4E12156D2292
:10145C00300715753801E53AB40105E5B120E6F61B
:10146C00120B2EC207E4F5380522D3E52294007442
:10147C008094884003E4F522E52270031215E122E2
:02008D00D3227C
:020DFE00D322FE
:02173700D322BB
:10131B0090E680E030E71590E6247402F0000000C0
:10132B00E490E625F0000000D2058013E490E6245B
:10133B00F000000090E6257440F0000000C205901C
:07134B00E6BAE0F539D322F8
:10169E0090E740E539F0E490E68AF090E68B04F0AE
:0216AE00D32245
:0817080090E6BAE0F526D322B9
:1016B00090E740E526F0E490E68AF090E68B04F0AF
:0216C000D32233
:02173900D322B9
:02173B00D322B7
:02173D00D322B5
:1001300090E6B9E0120F400156B301A1B5037DB6B8
:1001400003B8C003D8C10456C2049BC504FEC6054B
:100150002FC700000569E490E68AF090E68BF090E6
:10016000E6A0E020E1F990E68BE0F51800000090B1
:10017000E6047480F000000053297FAD29FF1211BE
:10018000C190E6047406F0000000E4F07F0AFE125D
:100190001297432980AD297F801211C1D207020531
:1001A0006BE490E68AF090E68BF090E6A0E020E128
:1001B000F990E68BE0F518D3943F4024E4F51974E8
:1001C000402519F582E434E7F583E0FF7400251932
:1001D000F582E43422F583EFF00519E519B440DF28
:1001E0007F8A7E001216C2902200E0FF7E00121667
:1001F000CC902200E0FF7E001216D6902200E0FF95
:100200007E001216E0902201E075F004A4FFAEF02B
:100210001216EA902201E075F004A4FFAEF0121667
:10022000F4902201E075F004A4FFAEF01216FE90E7
:100230002221E070035329BF902221E0B40103433F
:100240002940902205E0C3940250035329CF902205
:1002500005E0B40208E52954CF2410F529902205C1
:10026000E0B40308E52954CF2420F529902205E0C5
:10027000B40408E52954CF2430F529902239E070E0
:10028000035329F7902239E0B4010343290890224F
:1002900026E070055329FD8003432902902207E0E0
:1002A000FD7F401211C1902208E0FD7F201211C194
:1002B000902211E0FD7F101211C1902212E0FD7F0B
:1002C000081211C1902223E0F534902220E0F5338A
:1002D000902224E0F53B90222EE0F532902233E08C
:1002E000F531A3E0F53E90223AE0F542902206E097
:1002F000F530E530700375300190220BE0FEA3E08D
:100300007C002400F528EC3EF527A3E0FEA3E024C2
:1003100000F53DEC3EF53C902207E0FEA3E0240012
:10032000F52DEC3EF52CA3E0FEA3E02400F540EC17
:100330003EF53F902211E0FEA3E02400F537EC3EAD
:10034000F53690220FE0FEA3E02400F52BEC3EF5FD
:100350002A90222FE0FEA3E02400F525EC3EF524B0
:1003600090221DE0FD7F021211C190221EE0FD7F50
:10037000041211C190223FE0F54102056BE4F5192A
:1003800074002519F582E43422F583E0FF744025DA
:1003900019F582E434E7F583EFF00519E519B44067
:1003A000DF000000E490E68AF000000090E68B7425
:1003B00040F012154202056BA298E43390E740F03A
:1003C000A3E599F0000000E490E68AF000000090B8
:1003D000E68B7402F002056BE490E68AF090E68BFF
:1003E000F090E6A0E020E1F990E68BE0F518C298E5
:1003F000D39400500302056B90E740E0940A500745
:10040000E02430FF12008090E740E0B40A057F61ED
:1004100012008090E740E0B40B057F6212008090EC
:10042000E740E0B40C057F6312008090E740E0B441
:100430000D057F6412008090E740E0B40E057F65F3
:1004400012008090E740E0640F600302056B7F6656
:1004500012008002056B90E74074D5F0A3741EF083
:10046000A3740DF0A37478F0A3740AF0A3740EF0D3
:10047000E4A3F0A3F0A3F0300504A3F0800690E716
:100480004974FFF0000000E490E68AF0000000905C
:10049000E68B740AF012154202056B90E678E04490
:1004A00080F090E6797491F07F647E00121644909B
:1004B000E679E090E740F07F647E0012164490E613
:1004C00079E090E741F07F647E0012164490E6796F
:1004D000E090E742F07F647E0012164490E679E0F7
:1004E00090E743F090E678E04440F0000000E490AC
:1004F000E68AF000000090E68B7404F0806DE490D2
:10050000E68AF090E68BF090E6A0E020E1F990E634
:100510008BE0F518D39401405290E741E0FD7F4213
:1005200012156D90E740E0FD7F4E12156D803CE4A2
:1005300090E68AF090E68BF090E6A0E020E1F9905A
:10054000E68BE0F518D39400402190E740E070037B
:1005500012172F90E740E0B4010312173390E740E1
:0C056000E0B402071217608002D322C32F
:01056C00226C
:10161400C0E0C083C082D2015391EF90E65D7401B3
:08162400F0D082D083D0E03247
:10167200C0E0C083C0825391EF90E65D7404F0D065
:0616820082D083D0E032AB
:10168800C0E0C083C0825391EF90E65D7402F0D051
:0616980082D083D0E03295
:10135200C0E0C083C08290E680E030E70E8543475C
:10136200854448854B49854C4A800C854B47854CC2
:101372004885434985444A5391EF90E65D7410F0E5
:07138200D082D083D0E032DD
:10162C00C0E0C083C082D2035391EF90E65D740892
:08163C00F0D082D083D0E0322F
:10138900C0E0C083C08290E680E030E70E85434725
:10139900854448854B49854C4A800C854B47854C8B
:1013A9004885434985444A5391EF90E65D7420F09E
:0713B900D082D083D0E032A6
:01008F00323E
:01173F003277
:011740003276
:011741003275
:100F6600C0E0C0F0C083C082C0D075D000C000C051
:100F760001C002C003C004C005C006C007C2AFE579
:100F860038705090E678E04480F090E6797491F0FD
:100F96007F647E0012164490E679E090E7C0F07F09
:100FA600647E0012164490E679E090E7C1F07F6413
:100FB6007E0012164490E679E090E7C2F07F647EE8
:100FC6000012164490E679E090E7C3F090E678E0E8
:100FD6004440F090E7C0E538F000000090E68F74DA
:100FE60004F00000005391EF90E65FE04404F0D275
:100FF600AFD007D006D005D004D003D002D001D0A0
:0C10060000D0D0D082D083D0F0D0E032F7
:1010A500C0E0C0F0C083C082C0D075D000C000C011
:0D10B50001C002C003C004C005C006C00792
:1010C200C2AF90E6A1E020E1F990E780E0FF700472
:1010D200F5238030BFFF07752300D2068026BFFEAE
:1010E2000890E781E0F53A801BE4FD7F9012156DD0
:1010F20090E782E0FD7F4212156D90E781E0FD7F6F
:101102004E12156D00000090E68DE4F05391EF90C1
:08111200E65FE04408F0D2AFF3
:10111A00D007D006D005D004D003D002D001D00029
:0B112A00D0D0D082D083D0F0D0E032D3
:011742003274
:011743003273
:011744003272
:011745003271
:011746003270
:01174700326F
:01174800326E
:01174900326D
:01174A00326C
:01174B00326B
:01174C00326A
:01174D003269
:01174E003268
:01174F003267
:011750003266
:011751003265
:011752003264
:011753003263
:011754003262
:011755003261
:011756003260
:01175700325F
:01175800325E
:01175900325D
:01175A00325C
:01175B00325B
:01175C00325A
:01175D003259
:01175E003258
:01175F003257
:10164400AD07AC06ED25E0FDEC33FCED4C6007ED99
:071654001D70011C80F5224E
:060D5B008C1A8D1BA90794
:100D6100530107C2A77F0A7E00121644E4FBFAC3AF
:100D710074029BFFE9A807088002C313D8FC30E086
:100D810004D2A68002C2A67F0A7E00121644D2A512
:100D9100121644C2A51216440BBB00010AEB6403F0
:100DA1004A70CCE4FAFBC374099BFFE51BAE1AA899
:100DB10007088005CEC313CE13D8F930E004D2A6BC
:100DC1008002C2A67F0A7E00121644D2A5121644E2
:100DD100C2A51216440BBB00010AEB640A4A70C695
:0E0DE100D2A77F0A7E00121644C2A712164443
:010DEF0022E1
:0A16C200AD07AC06E4FF120D5B2239
:0A16CC00AD07AC067F04120D5B228F
:0A16D600AD07AC067F05120D5B2284
:0A16E000AD07AC067F06120D5B2279
:0A16EA00AD07AC067F01120D5B2274
:0A16F400AD07AC067F02120D5B2269
:0A16FE00AD07AC067F03120D5B225E
:0411C1008F1DA905D0
:1011C500C2A47F017E00121644E4FBFAAF03E9A82E
:1011D50007088002C313D8FC30E004D2A68002C2FF
:1011E500A67F017E00121644D2A5121644C2A5128E
:1011F50016440BBB00010AEB64084A70CFE4FAFB06
:10120500AF03E51DA807088002C313D8FC30E0042E
:10121500D2A68002C2A67F017E00121644D2A51274
:101225001644C2A51216440BBB00010AEB64084A1A
:1012350070CEC2A4D2A47F017E00121644C2A412AD
:0212450016444D
:011247002284
:04171F0043B10122AF
:0417230053B1FE229E
:0417270043B10422A4
:04172B0053B1FB2299
:0717180012172312172B2208
:1015E10012171F7F127E001216441217231217279B
:0A15F10012164412172B12164422A2
:1015FB00E4FBFA1215E17F467E001216440BBB008A
:08160B00010ABA0CEEBB0EEB64
:0116130022B4
:04172F0053B17F2211
:0417330043B180221C
:10101200E533B4010353B1EF12172FE534706F7546
:101022002301902202E075F040A485F01CF51DAF6B
:10103200237E00AC1CAD1D120F07D3EF9400EE947B
:101042000040117FEF7E03121297E51D151D7002FD
:10105200151C80DB902203E0751C00F51DAF237E7A
:1010620000AC1CAD1D120F07D3EF9400EE940040AC
:10107200117F007E01121297E51D151D7002151CCD
:1010820080DB902204E0FF7E001212978009752314
:1010920001E523640160FA121733E533B401034317
:0210A200B1108B
:0110A4002229
:100B2E00C2A0C206E5317003121733E52B452A70B9
:100B3E00031215FB753802121012753803300603B6
:100B4E00020C52E4F518F519C3E5199528E5189528
:100B5E00275030E4F51AF51BC3E51B95307480F869
:100B6E00651A9850141215E17F467E001216440540
:100B7E001BE51B7002051A80DF0519E519700205C9
:100B8E001880C5E532D394004005AF32121596E4B5
:100B9E00F518F519C3E5199540E518953F5030C283
:100BAE00813080FDD281E4F51AF51BC3E51B95302B
:100BBE007480F8651A98500D1215E1051BE51B702F
:100BCE0002051A80E60519E5197002051880C5D2CE
:100BDE00A0E4F518F519C3E519953DE518953C50B7
:100BEE0030E4F51AF51BC3E51B95307480F8651AD1
:100BFE009850141215E17F467E00121644051BE52F
:100C0E001B7002051A80DF0519E5197002051880A0
:100C1E00C5E536FD7F401211C1E537FD7F2012116B
:100C2E00C1C2813080FDD281C2813080FDD281E58A
:100C3E002CFD7F401211C1E52DFD7F201211C11236
:040C4E001760D2A0B9
:010C5200227F
:10156D00AB05AE0790E678E04480F090E679EEF0BA
:10157D007F647E00121644EBF012164490E678E07C
:09158D004440F07F641216442270
:1012DD00E4FBFAEF75F010A4AAF0FB90E678E04479
:1012ED0080F090E6797418F07F647E00121644AF9A
:1012FD0002EFF07F64121644AF03EFF07F64121615
:0D130D004490E678E04440F07F64121644FE
:01131A0022B0
:011760002266
:10154200E4F51AF51BD2A07F327E00121297C2A0D8
:101552007F327E00121297051BE51B7002051AC32B
:0A1562009403E51A6480948040DBD6
:01156C00225C
:101596008F1C432904AD297F801211C1E51C600B05
:1015A600C2813080FDD281151C80F15329FBAD2903
:0615B6007F801211C1222A
:10165B00E490E608F075C83443985053877FC2ACCA
:07166B0075CBFF75CA642274
:0D008000309902C2998F993099FDC29922E2
:1014BB00E4F557F5582098220558E5587002055762
:1014CB00AE57FFE4FCFD7BFA7AFFF9F8C3120F1954
:0E14DB005004D2048004C20480DBC298AF9992
:0114E90022E0
:08171000E4F556D2E9D2AF2244
:1013C00090E678E020E6F9C2E990E678E04480F023
:1013D000EF25E090E679F090E678E030E0F990E6ED
:1013E00078E04440F090E678E020E6F990E678E096
:0613F00030E1D6D2E92233
:10142A00A90790E678E020E6F9E556702390E67879
:10143A00E04480F0E925E090E679F08D51AF03A908
:10144A00077552018A538954E4F555755601D3221A
:02145A00C322AB
:1013F600A90790E678E020E6F9E556702590E678AC
:10140600E04480F0E925E0440190E679F08D51AFA3
:1014160003A9077552018A538954E4F55575560395
:04142600D322C322E8
:03004B00020C5351
:100C5300C0E0C083C082C085C084C086758600C0E2
:100C6300D075D000C000C001C002C003C006C007D9
:100C730090E678E030E206755606020D3D90E67880
:100C8300E020E10CE55664026006755607020D3D4F
:100C9300E55624FE605F14603624FE7003020D2EB9
:100CA30024FC7003020D3A24086003020D3DAB528D
:100CB300AA53A954AF5505558F82758300120EB8F8
:100CC30090E679F0E55565517070755605806B9027
:100CD300E679E0AB52AA53A954AE558E82758300D0
:100CE300120EE5755602E5516401704E90E678E008
:100CF3004420F08045E55124FEB5550790E678E0A1
:100D03004420F0E55114B5550A90E678E04440F0EC
:100D130075560090E679E0AB52AA53A954AE558EAE
:100D230082758300120EE50555800F90E678E04446
:100D330040F075560080037556005391DFD007D0FD
:100D430006D003D002D001D000D0D0D086D084D03A
:080D530085D082D083D0E0328C
:03000000021135B5
:0C113500787FE4F6D8FD75815802117C2B
:100EB800BB010CE58229F582E5833AF583E02250EF
:100EC80006E92582F8E622BBFE06E92582F8E22239
:0D0ED800E58229F582E5833AF583E4932253
:100EE500F8BB010DE58229F582E5833AF583E8F043
:100EF500225006E92582C8F622BBFE05E92582C8EF
:020F0500F222D6
:100F0700EF8DF0A4A8F0CF8CF0A428CE8DF0A42EFE
:020F1700FE22B8
:100F1900EB9FF5F0EA9E42F0E99D42F0EC6480C84F
:060F290064809845F022EF
:100F2F00EB9FF5F0EA9E42F0E99D42F0E89C45F018
:010F3F00228F
:100F4000D083D082F8E4937012740193700DA3A340
:100F500093F8740193F5828883E473740293686054
:060F6000EFA3A3A380DF54
:10114100020807E493A3F8E493A34003F68001F2B5
:1011510008DFF48029E493A3F85407240CC8C333AF
:10116100C4540F4420C8834004F456800146F6DF7E
:10117100E4800B0102040810204080901248E47EB4
:10118100019360BCA3FF543F30E509541FFEE49373
:10119100A360010ECF54C025E060A840B8E493A33A
:1011A100FAE493A3F8E493A3C8C582C8CAC583CA65
:1011B100F0A3C8C582C8CAC583CADFE9DEE780BE1D
:011296000057
:00000001FF
